:020000040000FA
:0400000040EF01F0DC
:10000800D8CF00F0E0CF01F0026EE9CF03F0EACFDD
:1000180004F0FACF05F0FBCF06F0F2A818D0F2A250
:1000280016D0F292F2987AA68B94E80ECF6E900EC4
:10003800CE6E9E90CD809D987988799A79A407D0C4
:100048007ABA05D00D0E766002D0020E76269DA8EB
:100058001CD09EA81AD09D987ABA04D079A802D04C
:10006800798E13D06750E96E020E6824EA6EEFCFDE
:10007800ADFF7A8A672A000E6822676605D0020EED
:10008800686202D0676A686A71069DAA72D09EAAE1
:1000980070D0F2927988E80ECF6E900ECE6E9E9058
:1000A800CD80ABA203D0AB98AB8863D0ABA41CD0F7
:1000B800AE50E20ECF6EB40ECE6E9E90CD8079AC6F
:1000C80004D04A0EAF6E799C54D07AAA52D07A9A4C
:1000D800798E7C0EAF6EAD6A798CD60ECF6EFC0E23
:1000E800CE6E9E90CD8045D001EE80F06650E92618
:1000F800AECFEFFF79AC04D04A0EAF6E799C2FD00B
:100108007AAA2DD06D50E96E020E6E24EA6EEFCFFA
:100118007BF001EE80F06650E926EF507B6213D049
:100128006D2A000E6E226D6605D0020E6E6202D038
:100138006D6A6E6A716605D07A9A7994766AF288E1
:100148000ED09D880CD07A9A798E7C0EAF6EAD6AEF
:10015800798CD60ECF6EFC0ECE6E9E90CD805F0E43
:10016800736007D079BC05D0662A600E666201D03C
:10017800666A9EA053D09E9079A84CD07998F28850
:100188007AA68B8476C07CF07C467C467C44060F3D
:10019800F924D8B0FA2AF96EE80ECF6E900E36D050
:1001A800E90ECF6EBC0E32D0EA0ECF6EE80E2ED01E
:1001B800EC0ECF6E140E2AD0ED0ECF6E400E26D068
:1001C800EE0ECF6E6C0E22D0EF0ECF6E980E1ED0B4
:1001D800F00ECF6EC40E1AD0F10ECF6EF00E16D000
:1001E800F30ECF6E1C0E12D0F40ECF6E480E0ED04A
:1001F800F50ECF6E740E0AD0F60ECF6EA00E06D096
:10020800F70ECF6ECC0E02D0F80ECF6ECE6ECD802C
:10021800798A04D079AA02D0799ACD909EA21ED06C
:100228009E922682572A130E576418D0576A26843E
:10023800582A010E586402D0586A2686592A130E85
:1002480059640CD0596A26885A2A090E5A6406D06D
:100258005A6A268A5B2A0A0E5B605B6A05C0FAFF47
:1002680006C0FBFF03C0E9FF04C0EAFF025001C05B
:10027800E0FF00C0D8FF100081EC11F0B5EC11F0E0
:10028800FCEC11F000012FEC12F0F6EC12F0040077
:10029800D180F28CF28ECA8479B634D06550665C0F
:1002A800076E07AE02D0600E072607C073F007522C
:1002B80059E001EE80F06550E926EFAE1ED0800EC1
:1002C800096E010E0A6E65C00BF00C6A0BBE0C06B7
:1002D80007C00DF00E6A0DBE0E06600E0F6E106A96
:1002E80013EC0AF0726E72503DE0FF0A03E1D8EC9D
:1002F8000EF038D0F288798635D0D8EC0EF0072E7B
:10030800D8D730D001EE80F06550E926EF50830A47
:100318000BE0330A0CE0010A14E0030A16E0060AAF
:1003280018E05B0A19E01BD0A4EC0EF01AD0000EFE
:1003380086EC0CF00FC008F010C009F044EC0BF08C
:1003480010D0010E86EC0CF00CD0020E86EC0CF0EE
:1003580008D032EC10F005D027EC0FF002D0D8EC22
:100368000EF0799626A24ED1269279B44DD079B85E
:100378004BD06750695C076E68506A58086E08AEC3
:1003880002D0020E0826075008103EE06750E96EBA
:10039800020E6824EA6EEFAE2FD0096A020E0A6ECA
:1003A80067C00BF068C00CF007C00DF008C00EF075
:1003B8000F6A106E13EC0AF0716E715025E0FF0A97
:1003C80003E1E3EC0EF020D06750E96E020E6824DA
:1003D800EA6EB20EEF6203D0060E766E01D0766A30
:1003E80067C06BF068C06CF071C06FF067C06DF0EB
:1003F80068C06EF0798408D0E3EC0EF00706000EB2
:10040800085A07500810C2E179A419D079AE0BD068
:10041800799E6BC067F06CC068F06FC071F067C000
:100428006DF068C06EF07AA80AD079B808D079BAA9
:1004380006D00DEC13F079B802D079AA9D8810EE99
:10044800B0F0096A080E0960DDD0E6500F90E7BCED
:100458000F800F92E7BA0F82E6BED2D0EA6A470E43
:100468000924E96EEF50D8B4CBD024EE00F0200E6A
:100478000902F350D9260E6A010E0A6E0A52D8B440
:10048800B6D0EA6A470E0924E96E0A50EF14D8B4C8
:10049800A8D0EA6A470E0924E96E0A1CEF16DECFD7
:1004A8000DF0DECF0BF07AA22BD00FB229D00D3889
:1004B800030B5BE10FA006D00EA004D0020ED926D4
:1004C8000E2A92D0020EE15EE6CF07F0E6CF08F0E2
:1004D8000F94EA6A370E0924E96E0A50EF14D8A47B
:1004E8000F8408960FB40886100E146E1A901A928C
:1004F80007C015F008C016F00E5094EC0AF035D07D
:100508000F0E0B140C6E0B38070B0B6E0B5006E01E
:10051800010A04E0030A02E0010A65E10BC010F0D9
:100528000CC011F00DC012F00EC013F009C014F089
:100538000A5018EC09F006E3EA6A800E0924E96E0D
:100548000A50EF120B5203E0020E0B620ED00C524F
:100558000CE0EA6A2F0E0924E96E0A50EF1405E14F
:100568000FA003D0020ED9263ED0DE507AA204D0C6
:10057800C2BB02D0DE5037D0DEBE35D0D8900D32A7
:10058800D8900D32030E0D14010A05E0030A11E09C
:10059800010A20E028D0EA6A2F0E0924E96E0A50E1
:1005A800EF1421E0EA6AA00E0924E96E0A50EF125E
:1005B8001AD0EA6A2F0E0924E96E0A50EF1413E1E3
:1005C800E550E6BC10D0EA6AA00E0924E96E0A508C
:1005D800EF1209D0EA6AA00E0924E96E0A50EF1258
:1005E80002D0040ED9260E2AD8900A3647D709C059
:1005F80024F0EA6A2F0E0924E96EEF50F0EC10F0AF
:10060800092A20D726A476D02694040079A006D0FB
:100618005D2E04D07990000EE2EC07F081B008D08E
:100628007AA80DD0742A140E746209D07A9807D06B
:10063800746A7AB804D0756602D0010E756E755268
:100648000FE0752A330E75620BD0756AF29EF2922E
:10065800F288AB889E9A9D8A9D98AC8AF28E7A8899
:1006680010EEB0F0076A080E076044D0E650E6AE18
:100678003FD0EA6A370E0724E96EEFCF09F007503A
:10068800DCEC10F00A6EEA6A2F0E0724E96E0AC045
:10069800EFFFEA6A4F0E0724E96EEFCF0CF0EA6A23
:1006A800800E0724E96EEFCF0DF00A5009180B6E83
:1006B800010E086E085216E008500D1410E10C5097
:1006C8000B1408140CE0EA6A370E0724E96E085088
:1006D800EF1AEA6A470E0724E96E0850EF12D8901D
:1006E8000836E8D7EA6A4F0E0724E96E0BC0EFFF19
:1006F800072AB9D726A6CCD326960A6A080E0A6016
:1007080056D1EA6A980E0A24E96EEF50D8B44DD152
:1007180024EE00F0200E0A02F350D9260D90076A45
:10072800010E0B6E0B52D8B435D1EA6A980E0A2422
:10073800E96E0B50EF14D8B427D1DECF09F0DDCF26
:100748000CF00C38070B086E01EE00F0080E0A02D8
:10075800F3500724D890E834E926EE06000EEF5A45
:1007680001EE00F0080E0A02F3500724D890E8348E
:10077800E926EE50EF10D8A407D1E26AD8900A34DF
:10078800B10FE16EE7BED4D0E7AA17D0050ED9267F
:100798000C38F00B0C6E0F0EDF140C26050ED95E0C
:1007A80008C00EF00CC00FF007C010F00AC011F01E
:1007B8000B5088EC08F00D80E7D0EA6AA80E0A24EE
:1007C800E96E0B50EF1433E0EA6A980E0A24E96EDA
:1007D8000B1CEF16EA6A800E0A24E96E0B50EF1420
:1007E80013E008C010F00F0E0C14116E126A07C047
:1007F80013F00AC014F00B5018EC09F0EA6A800EE6
:100808000A24E96E0B1CEF16EA6AA80E0A24E96EA0
:100818000B1CEF16EA6A270E0A24E96E0B50EF123A
:10082800EA6AA00E0A24E96E0B50EF12ADD0085008
:10083800020A03E0030E08621CD0EA6A980E0A2432
:10084800E96E0B1CEF1608C010F00F0E0C14116E99
:10085800126A07C013F00AC014F00B5018EC09F024
:1008680006E3EA6A800E0A24E96E0B50EF120D8047
:1008780028D0085202E0082C24D0EA6A980E0A24EC
:10088800E96E0B1CEF16EA6A800E0A24E96E0B1C4F
:10089800EF16DFBC08D0EA6A2F0E0A24E96E0B1C9B
:1008A800EF160D800ED0EA6A370E0A24E96E0B5057
:1008B800EF1407E1EA6A2F0E0A24E96E0B1CEF1603
:1008C8000D807AB261D0030ED926DFBE2ED0D89023
:1008D8000932D89009320914010A05E0030A11E027
:1008E800010A1DE022D0EA6A2F0E0A24E96E0B5095
:1008F800EF141BE0EA6AA00E0A24E96E0B50EF120F
:1009080014D0EA6A2F0E0A24E96E0B50EF140DE199
:10091800EA6AA00E0A24E96E0B50EF1206D0EA6AC2
:10092800A00E0A24E96E0B50EF12030ED95E2CD0EC
:10093800EA6A980E0A24E96E0B1CEF16EA6A270E7B
:100948000A24E96E0B50EF12EA6AA80E0A24E96E2F
:100958000B50EF1413E0EA6AA80E0A24E96E0B1C88
:10096800EF16EA6AA00E0A24E96E0B50EF12EA6A43
:10097800800E0A24E96E0B1CEF1606D0EA6A470EB1
:100988000A24E96E0B50EF12040ED926072AD890D4
:100998000B36C8D60DA009D00AC024F0EA6A2F0E7B
:1009A8000A24E96EEF50F0EC10F00A2AA7D610EEF0
:1009B800B0F00D6A080E0D6082D1D8900D340F6E1C
:1009C800E6CF07F0E6CF08F008AE77D16750695C4C
:1009D800096E68506A580A6E0AAE02D0020E0A26DC
:1009E800EA6A470E0D24E96EEF50D8B466D10ABE04
:1009F80006D0C00E095C010E0A58D8B05ED124EEAC
:100A080000F0200E0D02F350D926040ED95E000E18
:100A1800DA5A1068010E0E6E0E52D8B44ED1040E7A
:100A2800D926000EDA22102AEA6A470E0D24E96E4A
:100A38000E50EF14D8B43ED1EA6A470E0D24E96E81
:100A48000E1CEF16DECF0BF0DDCF0CF01290EA6A29
:100A5800370E0D24E96E0E50EF14D8A412800896B4
:100A680012B008860B38030B37E17AB2F4D0089835
:100A780012B00888EA6A270E0D24E96E0E50EF14AA
:100A8800D8B48BD0EA6A270E0D24E96E0E1CEF1637
:100A98000896EA6A3F0E0D24E96E0E50EF14088896
:100AA800D8B408980BC014F01A901A9207C015F021
:100AB80008C016F0105094EC0AF0EA6AA00E0D2453
:100AC800E96E0E50EF14D8A4F5D0EA6A800E0D2412
:100AD800E96E0E1CEF16EED00C38070B5EE17AB209
:100AE8005CD0EA6A270E0D24E96E0E50EF1416E06A
:100AF800EA6A270E0D24E96E0E1CEF16EA6A880EC4
:100B08000D24E96E0E50EF14D880D8B4D89003E2C3
:100B180012B0D0D042D012B040D0CCD0EA6A980EF1
:100B28000D24E96E0E50EF1422E1EA6A880E0D24B6
:100B3800E96E0E1CEF1612A010D00E50EF12030E25
:100B48000B14030A2AE00CC014F010C015F00DC0F5
:100B580016F00E50DEEC09F0ADD00CC014F010C049
:100B680015F00DC016F00E50DEEC09F0A3D0EA6ABD
:100B7800880E0D24E96E0E50EF14D880D8B4D890A2
:100B880003E212B003D009D012B007D0EA6A980E77
:100B98000D24E96E0E1CEF168DD0030E0B14010AFE
:100BA80007E0030A08E0010A08E0030A54E005D058
:100BB80012B003D050D012B04ED00B38030B40E126
:100BC800EA6A980E0D24E96E0E50EF1473E1EA6A92
:100BD8003F0E0D24E96EEFCF11F008AC03D00E5094
:100BE800111A07D010A003D00E50111202D00E1CFB
:100BF80011160E5011140888D8B40898EA6A3F0EE6
:100C08000D24E96E11C0EFFF0C38070B020A09E149
:100C18000CC014F010C015F00DC016F00E50CADB51
:100C280008D0200E146E10C015F00DC016F00E502E
:100C3800C1DB0886EA6A800E0D24E96E0E50EF12B9
:100C48000BC014F01A901A9207C015F008C016F0DD
:100C5800105094EC0AF07AA202D0C2AB2BD0D890F4
:100C68000B32D8900B32030E0B14010A07E0030A6B
:100C780008E0010A08E0030A1DE005D012B003D01D
:100C880019D012B017D0EA6AA00E0D24E96E0E50E2
:100C9800EF12030ED926000EDA22DF38030B06E125
:100CA800EA6A800E0D24E96E0E50EF12030ED95E2B
:100CB800000EDA5AD8900E36AFD60D2A7BD60E6AB9
:100CC800080E0E60D5D06750695C096E68506A5886
:100CD8000A6E0AAE02D0020E0A26EA6AA00E0E2496
:100CE800E96EEF50D8B4C2D00ABE06D0E00E095C57
:100CF800010E0A58D8B0BAD0E26AD8900E34B10FB3
:100D0800E16E24EE00F0200E0E02F350D926116A8F
:100D1800010E0F6E0F52D8B4A9D0EA6A470E0E24FE
:100D2800E96E0F50EF14D8A49BD0EA6AA00E0E24E7
:100D3800E96E0F50EF14D8B493D0E7AE08D0EA6A42
:100D4800980E0E24E96E0F50EF14D8A48CD0EA6ADE
:100D5800A00E0E24E96E0F1CEF16DECF0BF0DECFCF
:100D68000DF0DECF07F0DECF08F0040ED95E08C024
:100D78000CF00898EA6A370E0E24E96E0F50EF144B
:100D8800D8A408880C38030B61E1EA6A270E0E2400
:100D9800E96E0F50EF1408E0EA6A270E0E24E96E98
:100DA8000F1CEF16089844D0E7AE33D00B38030B6E
:100DB800020A03E0020A12E02CD0EA6A3F0E0E246F
:100DC800E96E0F1CEF16E7AC24D008A822D0EA6A17
:100DD8003F0E0E24E96E0F50EF121BD0030E0B14BA
:100DE80018E1EA6A3F0E0E24E96EEFCF12F0E7AC85
:100DF80003D00F50121A07D011A003D00F501212AF
:100E080002D00F1C1216EA6A3F0E0E24E96E12C0B9
:100E1800EFFF200E146E11C015F00EC016F00F5023
:100E2800C9DA0888EA6AA80E0E24E96E0F50EF1294
:100E3800E7AE07D0EA6A3F0E0E24E96E0F50EF14B2
:100E480001D0000E000A088AD8B4089A0CC014F021
:100E58001A901A8207C015F008C016F0115060DB0E
:100E6800040ED926112AD8900F3654D70E2A28D71F
:100E78007AA20ED0076A080E076007D0EA6A470E02
:100E88000724E96EEF10072AF6D7FF0AD8A47A924A
:100E980026A862D026985E520DE05E060F0E5E14FC
:100EA80009E15E3A5E060F0E5E1403E0140E86D862
:100EB8005E8A5E3A5F5206E05F2E04D0640E7ED8EA
:100EC8000A0E5F6E7AA42CD077060F0E771428E1ED
:100ED800773A0F0E7714076E080E07601DD0010EC3
:100EE800086E075005E0096ED8900836092EFCD721
:100EF8000850601407E0EA6A470E0724E96EEF68B5
:100F08007A8208D0C2A906D0EA6A470E0724E96E99
:100F1800EF687A82772A01D07A94773A0A0E7712A4
:100F280082B219D05C2A7AB607D00A0E5C620BD05E
:100F38007A86010E5F6E07D0020E5C6204D07A9644
:100F48005F6A650E5C6E640E5C6203D0D19000EF40
:100F580000F0000101D05C6A26AA50EF01F0269A41
:100F680026AC50EF01F05B04076E080E076050EFE7
:100F780001F0E26AD8900734B10FE16EE7AE0FD006
:100F880007506124196E000E62201A6EEA6A3F0E3D
:100F98000724E96EEF5026EC11F050EF01F00750EE
:100FA8006124196E000E62201A6EEA6A370E072451
:100FB800E96EEF5026EC11F050EF01F0246E245248
:100FC80005E024C05DF079808B9001D08B80120001
:100FD8001D6E010EEA6E1CC0E9FF1D461D461D442C
:100FE800060FF924D8B0FA2AF96EEF6A000E00004D
:100FF8003BD00A0EEF6E000E37D0140EEF6E000EC7
:1010080033D0230EEF6E000E2FD0320EEF6E000E8F
:101018002BD0410EEF6E000E27D0500EEF6E000E53
:1010280023D0640EEF6E000E1FD07D0EEF6E000E03
:101038001BD0960EEF6E000E17D0C80EEF6E000E86
:1010480013D02C0EEF6E010E0FD0900EEF6E010E26
:101058000BD0F40EEF6E010E07D0580EEF6E020E95
:1010680003D0200EEF6E030EEC6E12001B6E010E05
:10107800EA6E1AC0E9FF1B461B461B44060FF924FB
:10108800D8B0FA2AF96EE80EEF6E030E3BD0DC0EEC
:10109800EF6E050E37D0D00EEF6E070E33D0B80EB8
:1010A800EF6E0B0E2FD0A00EEF6E0F0E2BD0880E0A
:1010B800EF6E130E27D0700EEF6E170E23D0280E8A
:1010C800EF6E230E1FD0E00EEF6E2E0E1BD0500ECB
:1010D800EF6E460E17D0C00EEF6E5D0E13D0300EB9
:1010E800EF6E750E0FD0A00EEF6E8C0E0BD0100E9B
:1010F800EF6EA40E07D0800EEF6EBB0E03D0600E0D
:10110800EF6EEA0EEC6E1200126EEA6A2F0E1124D0
:10111800E96EEFCF14F0105005E0176ED890143236
:10112800172EFCD7030E14160F14146214D0269031
:101138000FB426802F0E1124246E12500BEC11F0E0
:1011480026900FB626802F0E1124246ED8901234C4
:101158000BEC11F013D026900FB026802F0E11241F
:10116800246E12500BEC11F026900FB226802F0E31
:101178001124246ED89012340BEC11F011C024F015
:10118800EA6A2F0E1124E96EEF50F0EC10F00F38D8
:101198000F0B0F6E080E1102F3501024136EEA6A3B
:1011A800980E1124E96E121CEF160E50020A03E085
:1011B800010A19E02FD0D89013341C6E0F5008DFA5
:1011C80001EE00F0D8901334E926EECF15F0EECFFB
:1011D80016F0155016101EE0EA6A980E1124E96EF2
:1011E8001250EF1217D0D89013341A6E0F503EDFFA
:1011F80001EE00F0D8901334E926EECF15F0EECFCB
:1012080016F01550161006E0EA6A980E1124E96ED9
:101218001250EF1201EE00F0D8901334E92615C0F1
:10122800EEFF16C0EEFF1200156E105202E0102CF1
:101238000BD012BC09D0EA6A980E1424E96E155036
:10124800EF1402E0D8901200EA6A370E1424E96E0F
:101258001550EF14D8B48FD0080E1402F35013248D
:10126800166E105203E0020E106206D0D8901634A3
:101278001C6E1150ADDE0AD0104C03D0030E106264
:1012880005D0D89016341A6E1150F0DE01EE00F039
:10129800D8901634E926EECF18F0EECF19F010509A
:1012A800020A07E0010A10E0030A37E0010A40E0F9
:1012B80060D01850191008E1EA6A2F0E1424E96E5C
:1012C8001550EF12D8901200EA6A980E1424E96EAD
:1012D8001550EF144EE1EA6AA80E1424E96E155071
:1012E800EF1405E0090E185E000E195A06D0EA6AD6
:1012F8002F0E1424E96E1550EF1A01EE00F0D89065
:101308001634E92618C0EEFF19C0EEFFEA6A980EF7
:101318001424E96E1550EF122CD01850191008E15A
:10132800EA6A2F0E1424E96E1550EF12D8901200B5
:10133800EA6AA80E1424E96E1550EF1405E0090EA8
:10134800185E000E195A06D0EA6A2F0E1424E96EA8
:101358001550EF1201EE00F0D8901634E92618C0A7
:10136800EEFF19C0EEFFEA6A980E1424E96E1550D4
:10137800EF12D88012001050020A07E0010A05E0B7
:10138800030A09E0010A07E013D0EA6A980E142458
:10139800E96E151CEF16EA6A980E1424E96E1550CA
:1013A800EF1406E1EA6A2F0E1424E96E151CEF16F5
:1013B800D8901200176E0F0E1414186E1438070BFD
:1013C800196E020A02E0196629D0080E1602F350B7
:1013D80015241A6E185206E0D8901A341C6E18504C
:1013E800F7DD16D0020E196209D001EE00F0D89090
:1013F8001A34E926090EEE6EEF6A0AD0196608D08B
:1014080001EE00F0D8901A34E926010EEE6EEF6A6C
:10141800EA6A980E1624E96E1750EF1212000B5064
:101428000924E96E0C500A20EA6EEFCF12F012ACD4
:101438002DD012AA28D00D06000E0E5A0D500E10EF
:1014480021E00BC013F00CC014F0132A000E142274
:1014580013500F6205D01450106202D0136A146A38
:1014680013500924E96E14500A20EA6EEFCF11F0E8
:10147800030E116402D0110E1160FF0C0D2A000E2C
:101488000E220BD0000C060E116E07D012AA03D044
:10149800040E116E02D0020E116E126A0B5009244E
:1014A800E96E0C500A20EA6EEF50121A0B2A000E51
:1014B8000C220B500F6205D00C50106202D00B6A40
:1014C8000C6A1104136E135226E00D06000E0E5A14
:1014D8000EBE03D00D500E10D8B4000C0B500924CA
:1014E800E96E0C500A20EA6EEFBEFF0C0B5009247F
:1014F800E96E0C500A20EA6EEF50121A0B2A000E01
:101508000C220B500F6205D00C50106202D00B6AEF
:101518000C6A1306D8D7123C02D011501200FF0CE7
:10152800176E1438030B186E1AB249D01A9416BCE9
:101538001A841F0E1616185005E0010A10E0030A57
:1015480030E03CD01AA405D017501526000E1622FC
:1015580067D0D89017301526000E162261D01AB41D
:1015680005D017501526000E162205D0D890173032
:101578001526000E16221AB009D0169A169816B615
:101588001688168616A84CD016964AD01688168A3B
:101598001AA446D0010E171617501688D8B41698F4
:1015A8003FD0168AD89017301526000E1622010E45
:1015B800171617501688D8B4169832D012003F0E56
:1015C8001616185005E0010A0EE0030A1DE027D0A0
:1015D800169616B81686169816BA1688100E14BCE3
:1015E800161A169A1DD0100E14BC161A169616B88E
:1015F80016861AB006D0169A168616A811D0169610
:101608000FD01688168A0CD0163416321532169852
:10161800D8B01688168A080E14BC161A01D0120003
:10162800D89015361636D8901532196A6950E96E71
:10163800020E6A24EA6EB00E1810EF6E1950D0DB55
:10164800196E6950E96E020E6A24EA6E15C0EFFF42
:101658001950C6DB196E6950E96E020E6A24EA6EEB
:1016680016C0EFFF1950BCDB196E6950E96E020E07
:101678006A24EA6E191CEF6E000EB2DB140E9ED4BB
:1016880008500914FF0AD8B4120010EEB0F00D6A21
:10169800080E0D6038D0E6CF0AF0E6CF0BF00BAE9F
:1016A80030D00BAC2ED0070E0B1624EE00F0200E17
:1016B8000D02F350D926106A010E0E6E0E5221E06B
:1016C800DFCF0CF00C38030B13E108500A6210D07E
:1016D80009500B620DD001EE80F06550E926269086
:1016E800EFBA26803F0E0D24246E0E500BEC11F03D
:1016F800040ED926102A0A2A000E0B22D8900E367C
:10170800DDD70D2AC5D712001C6ED9CF21F0DACF4C
:1017180022F024EE00F0200E1B02F350D926040E0E
:101728001A02F350D926DECF1EF023B01DD01E3882
:10173800030B1962E2D0195005E123A2DED02392EF
:1017480023B42382269023B22680370E1B24246ECE
:101758001C500BEC11F0EA6A470E1B24E96E1C5072
:10176800EF12140E2BDCC9D01966C7D023A2C5D03E
:101778001AB007D0EA6A980E1B24E96E1C1CEF16F3
:1017880008D0EA6A980E1B24E96ED8901C30FF0A2C
:10179800EF161AB027D0268023B42690370E1B24C4
:1017A800246E1C500BEC11F0268023B426902F0ECB
:1017B8001B24246E1C500BEC11F0269023B42680B9
:1017C800370E1B24246ED8901C340BEC11F0269095
:1017D80023B426802F0E1B24246ED8901C340BECC7
:1017E80011F07FD023B41FD02690370E1B24246E0F
:1017F8001C500BEC11F026902F0E1B24246E1C504D
:101808000BEC11F02690370E1B24246ED8901C3058
:101818000BEC11F026902F0E1B24246ED8901C3050
:101828000BEC11F05ED0DFCF1FF01F5006E0050A69
:1018380004E00F0A02E0050A27E126901FB226807D
:10184800370E1B24246E1C500BEC11F026901FB28F
:1018580026802F0E1B24246E1C500BEC11F02690B2
:101868001FB02680370E1B24246ED8901C300BEC3A
:1018780011F026901FB026802F0E1B24246ED890BE
:101888001C300BEC11F02DD02680370E1B24246E53
:101898001C500BEC11F02680370E1B24246ED890B8
:1018A8001C300BEC11F0040ED95E5F0EDF1417E04C
:1018B800060E1A14206E080E1B02F35020241D6E0B
:1018C80001EE00F0D8901D34E926010EEE6EEF6AA5
:1018D800EA6A980E1B24E96ED8901C30EF12040EA9
:1018E800D9261BC024F0EA6A2F0E1B24E96EEF509C
:1018F800F0EC10F0140EE2EC07F021C0D9FF22C082
:10190800DAFF1200086E50DA01EE80F06550E92621
:10191800D890EF340F6E48DA01EE80F06550E92672
:101928000F0EEF14106ED89010320F3201EE80F0C7
:101938006550E9261590EFBC15800850020A05E0AD
:10194800030A08E0010A19E02DD015B02ED00F685F
:101958001068FF0C15B029D0EFBA02D0EFA804D058
:10196800EFAA05D0EFA803D00F681068FF0CEFAA04
:1019780002D0EFA8EF88EF8C18D015A003D00F681D
:101988001068FF0CF80E0F5C030E10580EE3FC0EE7
:101998000F5C030E105809E20FC016F010C017F0C4
:1019A800D6D903D00F681068FF0C10EEB0F0096AA2
:1019B800080E0960C3D1E6CF11F0E6CF12F012BECF
:1019C800BBD124EE00F0200E0902F350D926DD50D9
:1019D800159612BA1586159A12BC158A070E121694
:1019E8000E6A0850010A06E0010A04E0020AD8B4A7
:1019F800EDD0A2D1010E0D6E0D52D8B49DD1DCCF21
:101A08000BF00F50116258D01050126255D001EEF1
:101A180080F06550E9261592EFB8158201EE80F046
:101A2800E9261594EFBA1584086607D0040EDFBEC0
:101A3800151A159C15B4158C06D0020EDFBE151AA2
:101A4800159C15B2158C030E0B14010A07E0030A46
:101A580008E0010A08E0030A2FE005D015BC03D00E
:101A68002BD015BC29D015B616D015AA14D00EA0A7
:101A780012D008C019F0239015B62380239215B20E
:101A88002382238415B423940EC01AF009C01BF0D6
:101A98000D503ADE11D008C019F0239015B62380F6
:101AA800239215B22382239415B423840EC01AF00E
:101AB80009C01BF00D5028DE030ED926DFAE77D003
:101AC800300EDF140C6E0C38086271D0070EDD146E
:101AD800146EDECF13F00F50136269D010501462E9
:101AE80066D001EE80F06550E9261592EFB81582B0
:101AF80001EE80F0E9261594EFBA1584086607D040
:101B0800040EDFBC151A159C15B4158C06D0020EF0
:101B1800DFBC151A159C15B2158CD8900B32D890CD
:101B28000B32030E0B14010A05E0030A06E0010A52
:101B380006E03DD015BC03D03AD015BC38D0D890BB
:101B48000B32D8900B32030E0B160B5007E0010A2C
:101B580002E0030A2CE1159215B4158215B616D0C9
:101B680015AA14D00EA012D008C019F0239015B6EB
:101B78002380239215B22382238415B423940EC0A4
:101B88001AF009C01BF00D50BFDD11D008C019F0C4
:101B9800239015B62380239215B22382239415B47B
:101BA80023840EC01AF009C01BF00D50ADDD0E2ABB
:101BB800112A000E122215AA06D015B604D00EA0BE
:101BC80002D01106125AD8900D3616D7010E0D6E96
:101BD8000D52D8B4B1D00F5011623FD010501262DC
:101BE8003CD0DCCF0BF001EE80F06550E926159271
:101BF800EFB81582020EDFBE151ADD50030E0B1466
:101C0800010A07E0030A08E0010A08E0030A25E0E0
:101C180005D015B203D021D015B21FD001EE80F047
:101C28006550E926EFAA03D00E2AD8900D3608C0D1
:101C380019F02390239215B2238223940EC01AF030
:101C480009C01BF00D5060DD01EE80F06550E926FB
:101C5800EFAA03D00E06D8900D321598DCCF0BF002
:101C6800030ED926000EDA22DFAE5CD0300EDF1468
:101C78000C6E0C38086256D00F0EDD14146EDECFD1
:101C880013F0D890143213320F5013624BD0105007
:101C9800146248D0DD5001EE80F06550E926EFBAB5
:101CA80003D0DEA003D03ED0DEA03CD001EE80F011
:101CB8006550E9261592EFB81582020EDFBC151A99
:101CC800D8900B32D8900B32030E0B14010A05E0A2
:101CD800030A06E0010A06E025D015B203D022D097
:101CE80015B220D0D8900B32D8900B32030E0B16B9
:101CF8000B5005E0010A07E0030A05E013D015942C
:101D080015B2158415820BC019F02390239215B2D1
:101D18002382239415B423840EC01AF009C01BF043
:101D28000D50F2DC0E2AD8900D36157815B896D7D6
:101D3800112A000E12224CD7092A3AD60F50120047
:101D480033D8C2A503D07A840A0E776E1200C2A7D0
:101D58002AD001EE80F06550E926EFB824D0030EB2
:101D68001614196E01EE80F06550E926EFBA198451
:101D7800080E196018D0E26AD8901934B10FE16ED4
:101D8800C2A709D0E7AE0FD0EA6A470E1924E96E58
:101D9800EF687A8208D0C2A906D0EA6A470E1924E9
:101DA800E96EEF687A82120001EE80F06550E9264C
:101DB800EF6A652A600E656201D0656A1200675095
:101DC800E96E020E6824EA6EEF6A672A000E68223E
:101DD800676605D0020E686202D0676A686A1200F8
:101DE8001B6E6950E96E020E6A24EA6EEF501B1AE8
:101DF800692A000E6A22696605D0020E6A6202D05C
:101E0800696A6A6A1B501200B00E126E136A146A6D
:101E1800B50E156E53DA116A106A040E10600ED0F2
:101E2800136E1150126E400E1124146EB50E156A01
:101E3800152244DA400E1126102AEFD7D9DA268E59
:101E48000ADB269E1200B0DFC2A31200ADDF01EE4E
:101E580080F06550E9267C0EEF6277D0A5DF01EEB1
:101E680080F06550E926EFCF0CF09EDF9DDF01EE94
:101E780080F06550E926EFCF09F096DF01EE80F09B
:101E88006550E926D890EF34086E093409320832D3
:101E98003F0EC0150B6EC1C00AF07AB606D00850C6
:101EA8000A6253D009500B6250D07EDF7DDFFC0EF2
:101EB8000C14200A0BE0080A09E0040A1AE04C0A8C
:101EC8002BE0080A29E00C0A34E03FD07AA60CD0AF
:101ED800C2AF07D00CC00DF008C00EF009C00FF05B
:101EE80035D8010E92D831D0C2AF2FD07F0E8DD801
:101EF8002CD07AB60CD00CC00DF008C00EF009C07A
:101F08000FF024D8C2AF21D0010E7FD81ED0C2AFA7
:101F18001CD07F0E7AD819D07AA606D0D0D8C2AFF6
:101F280014D0400E72D811D0C2AF0FD07F0E6DD82A
:101F38000CD07AB606D0C3D8C2AF07D0400E65D849
:101F480004D0C2AF02D07F0E60D8120015EE00F0A8
:101F5800E70EE66E0E0EE66E7C0EE66E0DC0E6FF30
:101F6800E66AD8900E360F36D8900E320FC0E6FFCC
:101F78000EC0E6FFE66A166A01EE80F06550E926B3
:101F8800EFCF14F014C018F018380F0B186E0CDFD0
:101F980001EE80F06550E926EFCF15F015C017F077
:101FA800179E14B0178E18500FE1160E17600CD03C
:101FB800B00E1724E96E000E1820EA6EEFCF16F067
:101FC800140EE2EC07F013D0160E175C010E185829
:101FD8000EE2160E175E000E185A1750E96E040E20
:101FE8001824EA6EEFCF16F0140EE2EC07F0149204
:101FF80016BE148214C0E6FF15C0E6FF7F0E161445
:10200800E66EE66AE66A7A8C12000D6E0E6A695010
:10201800E96E020E6A24EA6EB40EEF6E0E50E0DE30
:102028000E6E6950E96E020E6A24EA6E6F0EEF6E4C
:102038000E50D6DE0E6E6950E96E020E6A24EA6E04
:102048000DC0EFFF0E50CCDE0E6E6950E96E020E29
:102058006A24EA6E0E1CEF6E000EC2D6096AA4DE70
:1020680001EE80F06550E9266F0EEF6227D07AAC5A
:1020780025D07A9C15EE00F06950E96E020E6A24AC
:10208800EA6EE6CFEFFF0950ABDE096E020EE75CA1
:10209800086E6950E96E020E6A24EA6EE6CFEFFF19
:1020A80009509EDE096E082EF4D76950E96E020EBB
:1020B8006A24EA6E091CEF6E000E92D6120001EE39
:1020C80080F06550E926EFCF0FF06EDE01EE80F06C
:1020D8006550E926EFCF0EF00E9E0FB00E8E64DE2F
:1020E80001EE80F06550E926EFCF0DF00D9E0FB29E
:1020F8000D8E0F380F0B0F6E140E0E6202D00F529A
:1021080005E0150E0E620BD00F6609D0AA0E0D62FF
:1021180001D07ADEA10E5E6E140EE2EF07F00F50CA
:1021280019E1140E0E6016D0120E0E6203D00F5273
:10213800D8B40D82B00E0E24E96E000E0F20EA6EA0
:102148000DC0EFFF04000EC019F00FC01AF00D50BB
:1021580079D81BD0160E0E5C010E0F5815E2160E1C
:102168000E5E000E0F5A0E50E96E040E0F24EA6E32
:102178000DC0EFFF0400400E0E24196E000E0F2054
:102188001A6E0D505FD801D0120032D92BDA0F50D9
:102198000AE1100E0E6007D0010E0E14010A03E1C9
:1021A800268E59D9269E510E5E6E140EE2EF07F068
:1021B800196EF00E801619508026899881CF1AF072
:1021C8001A9082BA1A808988EA6A900E1924E96EF0
:1021D800EF501A1A1A501200256EEA6A900E24243B
:1021E800E96EEF50251A010E9316949A25C081FFC7
:1021F80025A0829A25B0828AF00E8016080E242423
:10220800802689988988FE0E9312948A1200256E7A
:1022180024C0E9FFEA6AD890EF14D8A4D88026A091
:1022280003D02550EF1202D0251CEF161200A6B2DB
:10223800FED71CC0A9FF1DC0AAFFA69EA69CA6800B
:10224800A85012001B6E19C01CF01AC01DF0EFDF59
:102258001B1832E0A6B2FED71BC0A8FF19C0A9FF01
:102268001AC0AAFFA69EA69CA684F29E550EA76E2B
:10227800AA0EA76EA682F28EA694632A000E642286
:10228800E90E635C030E64580EE3636A646A612AAC
:10229800000E6222F10E615C030E625804E3400EE8
:1022A800616E010E626E19C01CF01AC01DF0BFDF0E
:1022B8001B1802E0D8901200D8801200A68EA69CA7
:1022C800F86A1550F76EC00E1414F66E12C0E9FFC6
:1022D80013C0EAFF400E166E0900F552F5CFEEFF67
:1022E800162EFAD712000AC0F6FF0BC0F7FFF86ADD
:1022F800A68EA69C0800F55012000F0EC16E070EA0
:10230800B46E300E806EC00E926E816A9368D50EE0
:10231800826EEA0E946ED0A60AD0D0A408D000EE41
:1023280000F00F0EEE6AEA62FDD7E9AEFBD7F19C2A
:10233800F298F2924A0EAF6EAC84AC98AB8E9D9830
:102348009D9AAC9AAB98D56ACD6A9E909D80480EAE
:10235800CA6ECC6A7C0ECB6E9E929D82180EB16EB0
:102368001200140E0A6EB50E0B6EBDDF096E140E48
:102378001C6E1D6A5CDF091809E009C0A8FFA68465
:10238800550EA76EAA0EA76EA682A69400EEB0F010
:10239800076A086AA68407C01CF008C01DF047DF5A
:1023A800EE6E550EA76EAA0EA76EA682072A000E1D
:1023B8000822085003E1150E0764EDD704EE00F07B
:1023C800400E076E086A07C01CF008C01DF02FDF1A
:1023D800EE6E550EA76EAA0EA76EA682072A000EED
:1023E8000822400E075C010E0858EDE3A69412007F
:1023F8006068010E126E10EEB0F0136A080E1360DA
:1024080029D0EA6A900E1324E96EEF6A010E156E60
:1024180024EE00F0200E1302F350D926E650E6BE53
:1024280003D0D92A121C6016176A200E17600ED026
:10243800DFAE06D0EA6A900E1324E96E1550EF124B
:10244800D8901536040ED9261726EFD7D89012360D
:10245800132AD4D71200010E9316949A60C081FFF4
:1024680060A0829A60B0828A899A898AFE0E931245
:10247800948A8B981C6E030E1D6ED9DE616E1C68E3
:10248800030E1D6ED4DE626E1890F10E615C030EB1
:10249800625805E31880400E616E010E626E269C3C
:1024A800C2B1268C26AC15D026AE05D061C016F078
:1024B80062C017F005D06128166E000E6220176EF4
:1024C800F10E165C030E175804E3400E166E010E4B
:1024D800176E070E126E12BE74D0E26AD8901234CC
:1024E800B10FE16E26AC60D018B002D026AE02D093
:1024F800136A0AD0125061241C6E000E12BEFF0E21
:1025080062201D6E94DE136E040012501624196E9C
:10251800000E12BEFF0E17201A6E135093DEE7BE90
:102528003DD0EA6A370E1224E96E13C0EFFFE7AA1E
:102538002FD0EA6A2F0E1224E96E13C0EFFF12C0E3
:1025480024F0EA6A2F0E1224E96EEF5045DE020EDF
:10255800156E010E146E080E146026D0030E1314A7
:10256800030A0BE1196A23802382238414C01AF01A
:1025780012C01BF0155088EC0BF0D8901332D8908D
:102588001332D8901536D8901536020E1426E3D794
:10259800EA6A470E1224E96EEF6806D0EA6A3F0E2F
:1025A8001224E96E13C0EFFFE7AE09D0125000DE27
:1025B800136EEA6A370E1224E96E13C0EFFF120693
:1025C8008AD716C061F017C062F00400FE0E196EBB
:1025D800030E1A6E615036DE04001968030E1A6E77
:1025E800625030D6706A106A080E106009D0DA6A34
:1025F800D8901034B00FD96EDF507026102AF4D757
:10260800040EC103F35070263F0E701670C0C3F05D
:102618001200096A705009600ED0A192B368140EB6
:10262800B26EB180A1A2FED7B19079B804D079BAC0
:0826380002D0092AEFD71200BD
:10B50000008008801080188020802880308038805B
:06B51000E7100B000857D4
:10B54000230000002300000023000000230000006F
:10B55000230000002300000023000000230000005F
:10B56000230000002300000023000000230000004F
:10B57000230000002300000023000000230000003F
:10B58000230000002300000023000000230000002F
:10B59000230000002300000023000000230000001F
:10B5A000230000002300000023000000230000000F
:10B5B00023000000230000002300000023000000FF
:10B5C00023000000230000002300000023000000EF
:10B5D00023000000230000002300000023000000DF
:10B5E00023000000230000002300000023000000CF
:10B5F00023000000230000002300000023000000BF
:10B6000023000000230000002300000023000000AE
:10B61000230000002300000023000000230000009E
:10B62000230000002300000023000000230000008E
:10B63000230000002300000023000000230000007E
:020000040020DA
:080000000507000B00010001DF
:020000040030CA
:08000000FF021F08FF8181FFD0
:00000001FF
